:020000040000FA
:090000000219FD858A6502040A5B
:03000B000215B02B
:0500130002041601FFCC
:0F001B003034F8B285C574C8868BC804C57432FA
:03002B000203E2EB
:03003B000215307B
:03005B0002042577
:10007300C2AF53E67F7592FA7593FFD2AF53917F68
:0C008300302D08C22D303B0302157032F6
:1000B0004A45534330312023323420202020202051
:1000C0000406080C10182030406080A0C0C2AFC0E9
:1000D00082C083901480E493B4541BA3E493B44C83
:1000E00015A3E493B4580FA3A3A3E493B404071295
:1000F0001500D23B8002C23BD083D082D2AF22C255
:10010000AFC2A8C2CAC28EC0D075D008A8CCA9CD33
:10011000D2CAD2AF53E6EF85618BC0E0C0F0758ADA
:1001200000C3E89562F8E99563F9C3E913F9E813A8
:10013000F8E97021E89573401C95735018E582B476
:1001400010137C007B007A007908900000A860C33F
:10015000E813F8215E900000D2A8D2AA6134E0FD35
:10016000C39CC39840EF98EB33FB0582E0FCC39D32
:10017000C39840E198EB33FB0582E0FDC39CC39834
:1001800040D398EB33FB0582E0FCC39DC39840C588
:1001900098EB33FB0582E0FDC39CC39840B798EB16
:1001A00033FB0582E0FCC39DC39840A998EB33FB69
:1001B0000582E0FDC39CC398409B98EB33FB05820E
:1001C000E0FCC39DC398408D98EB33FB058221D999
:1001D000900000D2A8D2AA6134E0FDC39CC398402D
:1001E000EF98EA33FA0582E0FCC39DC39840E1989A
:1001F000EA33FA0582E0FDC39CC39840D398EA3302
:10020000FA0582E0FCC39DC39840C598EA33FA051D
:1002100082E0FDC39CC39840B798EA33FA0582E0B8
:10022000FCC39DC39840A998EA33FA0582E0FDC358
:100230009CC398409B98EA33FA0582E0FCC39DC3B7
:1002400098408D98EA33FA0582EBC46B6A54F0F952
:10025000EAC4303301F454F0C3996009900000D22D
:10026000A8D2AA6134D2C0EBF4C454F0F9EAF4C4C1
:10027000540F49FAEBF4C4540FFBC3EAF99460FA43
:10028000EB9400FB5020C3E97B007A0079006016F4
:10029000C3135006F9C3954D600AE9F54D754E003C
:1002A00079008002054E303A27C3EA94D0F8EB94E7
:1002B00007F9400BE8FAE9FB203109D23141C4309B
:1002C0003102C231203902B231C3EA33FAEB33FBD7
:1002D000EB2B3B3BF9C3EB13FBEA13FAEA29FAEBEE
:1002E0003400FB30E3047AFF7BFFE5255403601BF9
:1002F000202A18E55833F9EB7007C3E99A4002E960
:10030000FAE536C4332AFAEB3400FBC3EA33C454AB
:100310000FF8EB33C454F048F87005EA6002780136
:10032000900000E52260021522614A900000D2A8E8
:10033000D2AA61340522E52270021522C3E5229477
:1003400032500261BF754F0061C2884FD230E86001
:1003500003755000C3E556FC95574002AC57C3ECFB
:10036000954F5008EC75F008A4FAABF0EBF41313BA
:1003700092D5A2E75401F9EAF4FC13A2D513F8E5EB
:100380006423F564EC54032431835564600BE82442
:1003900001E9340020E10208F9C3E89419FAE9946C
:1003A00000FB50047A007B00885189528A538B5499
:1003B00075230A53F7DF43F740800700115577751F
:1003C000230AE5E6A2E082C0400ED2AAD2A8D0F06D
:1003D000D0E0D0D043E6103243E610D0F0D0E0D0E9
:1003E000D032C0D0C0E0C2CF053AE5236002152369
:1003F000C3E54F60057550008105E5502401F550B7
:1004000050037550FFD0E0D0D032C0E0E565856183
:100410008BF0A3D0E032C2AAD28EC2CA85CC62854C
:10042000CD63D2CA3253F7DFC0E0E5F9E5FA30E137
:100430000F8551E98552EA8553FB8554FC53F7BF7C
:10044000D0E0327901801879038014790A8010791C
:100450000F800C791E80087964800479C880007848
:100460001474F0000000D5E0FAD8F6D9F222790130
:10047000801479038010790A800C791E80087964D1
:10048000800479C880007591007594987595FC7505
:100490009104D22D43E680303B0953E67F302D0690
:1004A000121550202DFDD9DE2278FF20282879A1B1
:1004B000E76023E571601F74FF8571F0848539F072
:1004C00030290375F005A4F8C5F0600278FFC3E891
:1004D00095585002A858885722C3E57094E4E571F6
:1004E0009400E55750031481EA046002F557227521
:1004F000E890220559C3E5599408405330EDF4A81B
:10050000BDA9BE755900E9FA79A0E76041EA700615
:10051000E55A6018800CC3E8955A600EE55A5005FC
:10052000600A1480070460FA8002E55AF55AC39500
:100530005F401B7556C0C394044013755680C39426
:1005400004400B755640C39404400375560022E5E1
:10055000562410500274FFF55622743279A687F0A3
:10056000A4C5F0A2F733F558227570007571F0221A
:10057000C2AFC2CAA8CCA9CDAA3A30CF010AD2CA0A
:10058000D2AFC3EA13FAE913F9E813F8853B3E85C5
:100590003C3F883B893C8A3D22C2AFC2CAA8CCA955
:1005A000CDAA3A30CF010AD2CAD2AFAB3BAC3C881D
:1005B0003B893CC3E89BF8E99C202809F9302C03CF
:1005C0000206AC803FAD3D8A3DF9EA9DFA600678AF
:1005D000FF79FF8013AE3EAF3F8B3E8C3FA83BA917
:1005E0003CC3E89EF8E99FF9C3E57113FBE570137E
:1005F000FAE82AF570E93BF57150067570FF7571E0
:10060000FF020651AA70AB71AC70AD717E047F021F
:10061000C3EB9404400D1E1FC3EB94084005202932
:10062000021E1FC3ED13FDEC13FCDEF7C3EA9CFAB8
:10063000EB9DFBEF6009C3E913F9E813F8DFF7EA74
:1006400028FAEB39FB8A708B7150067BFF8B708B1D
:1006500071C3EB94025002D22C3028057F030206AE
:100660007D7892E6FFC3E537948240110FC3E537EA
:1006700094A040010FC3EF940640027F057E02E57F
:1006800071C4540FF9E571C454F0F8E570C4540F07
:1006900028F8C3E89EFAE99400FB4009C3EA9401F4
:1006A000EB940050047A01E4FB0206F8AA70AB71E7
:1006B000EBC4FEEAC4540F4EFCC3EA9CFAEB940070
:1006C000FBC3E813C313F8EA28FAEB3400FB8A7083
:1006D0008B71C3EB94024002C22C7802EBC4FE7B08
:1006E00000EAC4540F4EFAC3EA98FA4005C39401D5
:1006F00050027A017892E6FF303B0953E67F302DB5
:1007000006121550202DFD854992854A93D22D431E
:10071000E680C3E49AF8E49BF9302C03020790E8E2
:10072000FAE9FBD3E913FDE813FC8849894AC3EFD2
:1007300094036038EF20E00CE82CF8E93DF9ECFA7E
:10074000EDFB8013E828F8E939F9C3E82401F8E95A
:100750003400F97AFF7BFFC3EF9403400F8A4B8B81
:100760004C884589468C478D480207C5884B894C83
:100770008A458B468C478D48302812754BF0754C56
:10078000FF7547F07548FF7549F0754AFF0207C5C8
:10079000E8FAD3E813FC8849C3EF94036021EF2003
:1007A000E007E82CF8ECFAE1B0E8282401F87AFF39
:1007B000C3EF940340098A4B88458C470207C588DC
:1007C0004B8A458C47303B0953E67F302D06121586
:1007D00050202DFD753402D22D43E680E5255403CB
:1007E0006034A870A971C3E913F9E813F8C3E913D9
:1007F000F9E813F8302804E92440F9C2AF53E67F42
:10080000759100C3E498F594E499F595759104D237
:100810002D43E680D2AF22D22075440075200030EF
:100820002B03752040800ED2207544007520403087
:100830002B0375200078017901202C20E525540335
:100840006002C2207914E571C313700104F8C394E7
:100850001440027814302804781B791B202D11E5F0
:1008600044600D302803D53404D22101E41207D7A7
:100870000544E59B5440B52004D2A001CCC2A03071
:10088000280908C3E899400118015C20200B08C31F
:10089000E8994003020835015CC22053E67F759158
:1008A00000302C117594007595F8759104D22D4384
:1008B000E680020835E5717EFFC3334005C333404F
:1008C00001FEC3E49E759400F59501AAC3E5339437
:1008D000015003020835302003020835D80201E236
:1008E000015CC221C2A0C2AF53E67F759100854B67
:1008F00094854C95759104854592854693D22D43F8
:10090000E680D2AFE5255403600720290205338035
:100910001030210D202B0A2020071581158102118E
:100920004F2278003020027801E53775F007A4F9EE
:10093000E5F028F5F0E9A2F013A2F113A2F213F505
:1009400037C394785003753778C3E5379538400935
:10095000C291C293C29575D53F303B0953E67F30B3
:100960002D06121550202DFD854792854893D22DD6
:1009700043E68022203810C2AFC292D29075D50FC4
:10098000D2AF759F034144C2AFC292D29475D53C99
:10099000D2AF759F034144203810C2AFC29575D5C0
:1009A00033D290D2AF759F134144C2AFC29175D577
:1009B00033D294D2AF759F234144203810C2AFC2C6
:1009C00090D29475D533D2AF759F238077C2AFC2D2
:1009D00094D29075D533D2AF759F138067203810AD
:1009E000C2AFC29375D53CD294D2AF759F038054E9
:1009F000C2AFC29375D50FD290D2AF759F0380441A
:100A0000203810C2AFC294D29275D53CD2AF759F38
:100A1000138031C2AFC290D29275D50FD2AF759FFD
:100A2000238021203810C2AFC29175D50FD292D247
:100A3000AF759F23800EC2AFC29575D53CD292D2BE
:100A4000AF759F13227A1C7B3C80127A147B4B80FB
:100A50000C7A107B5A80067A0A7B788000E55BD599
:100A6000E001227902E4C292D5E0FDD293D5E0FD07
:100A7000C293D5E0FDD292D5E0FDE920E002D2910B
:100A800030E002D295E55BD5E0FDE920E002C291BD
:100A900030E002C2957496D5E0FDD9C9EAF8D5E0F8
:100AA000FDD8FBDBB8C29222C291C293C295C2901C
:100AB000C292C29475D53F22788076FF0876FF08EF
:100AC00076FF0876FF0876FF0876FF087609087635
:100AD000FF087601788C76010876FF0876FF0876A5
:100AE000FF0876FF0876FF0876030876FF0876FF92
:100AF0000876FF0876250876D0087628087650080C
:100B000076040876FF0876020876FF08767A08767B
:100B1000FF0876070876010876FF0876FF0876005A
:100B2000087600227888E6C39403D23A5002C23A8B
:100B3000C238E630E102D238A23892397886E6141B
:100B40009000C09378A6F67886E6F539C3940250F3
:100B500003753902789CE67538FFB402037538A036
:100B6000B4030375388278A0E6F860067428240977
:100B7000D8FCF55F2278A5E6F954037000E9540C1F
:100B80007000E954307000E954C0700022755D00B7
:100B9000755E007597DE7597AD7581C043FF8075F2
:100BA000EF0675A90075A90051A87580FF75F1F0D1
:100BB00075A4007580FF75D4FF75900075F23F75C0
:100BC000A53F75900075D53F75A00075A601E5B5E8
:100BD00025E0600975A71075CF0075A70075E34083
:100BE00075E20251A8E4F8F6D8FD51B812118578E3
:100BF00098865B753001756401C2AF12045B514584
:100C000012044F12044F12044F514B12044F12049E
:100C10004F12044F515112044F12044F12044F51FE
:100C20005751571204577175C2AF53A4DFD285755F
:100C30005D00755E00AAE475E4D578FA79FA30852E
:100C400009D9FBD8F7021C008AE4C2AF7124789856
:100C5000865B51A875C804759104C22D75D840757E
:100C6000D90875F781759E0375960175DB4275DAB3
:100C70004275A82175E61043B805759B80759D00E7
:100C800075D10C75BC5975BB1075E88075B2011231
:100C90000443900000758800757220753600C230DC
:100CA000754D00754E0075E45D1200CDD233758828
:100CB000517589AA758C00758D00C2A9D2ABD2AAD4
:100CC000D2AF758E017561C0756014757350752251
:100CD0000A1200CD12047E756010C3E522940A75D5
:100CE0004D00754E004077758E0C756180756028DB
:100CF00075732875220A1200CD12047E756020C318
:100D0000E522940A754D00754E00405275E4D5C237
:100D100033758E017561C075601475735075220A44
:100D20001200CD12047E756010C3E522940A754D41
:100D300000754E004028758E0C75618075602875B1
:100D4000732875220A1200CD12047E756020C3E557
:100D500022940A754D00754E004003020C281204BF
:100D600072203003020C28C2AFA233823B400651EE
:100D7000575157800451515151D2AF12048212047D
:100D80007EC3E54F9401400280EFC2AFA233823BA5
:100D9000401D5145D2AF12047EC2AF5145D2AF12B1
:100DA000047EC2AF5145D2AF12047EC2AF8006515D
:100DB0005751575157D2AF120482753000757000E9
:100DC000757100754000754100E4F531F53275200C
:100DD0000005203001477520000531E531F4703DF4
:100DE0000532789AE67819146012783214600D781A
:100DF0007D14600878FA146003753200C3E53298F8
:100E0000401B51A812044315327531007899865B56
:100E1000C2AF5157D2AF7898865B12047E12047627
:100E2000E5237002812812046E3030A5C3E54F948B
:100E300001500AC3E54D94015016020DD112047EF3
:100E4000E5237003020C28754D00754E00020FF06B
:100E5000C3E54D94017015C2AF51A87899865B51D6
:100E6000457898865BD2AF12047EE1E0C3E54D94ED
:100E7000027015C2AF51A87899865B514B7898865D
:100E80005BD2AF12047EE1E0C3E54D94037015C25E
:100E9000AF51A87899865B51517898865BD2AF1292
:100EA000047EE1E0C3E54D94047015C2AF51A8780B
:100EB00099865B51577898865BD2AF12047EE1E049
:100EC000C3E54D94057015C2AF51A87899865B5162
:100ED000577898865BD2AF12047EE1E0C3E54D946B
:100EE00007701AC3E54E94065002020E26740130B4
:100EF0003A0274037888F6C238C239E1E0C3E54D9E
:100F00009408701AC3E54E94065002020E2674022D
:100F1000303A0274047888F6D238D239E1E0C3E579
:100F20004D94097018C3E54E94065003020E263006
:100F30003A0BC37888E69402F6C23AE1E0C3E54D85
:100F4000940A7017C3E54E94065003020E26203A09
:100F50000A7888E62402F6D23AE1E0C3E54D94141B
:100F60007026C3E54E94065003020E26C2AF901AB7
:100F70000B740093D2AF7888F613C238C23940029E
:100F8000D2384002D2398058C3E54D94157038C329
:100F9000E54E94064050C2AF901A0B740093D2AF46
:100FA000F8B801027402B802027401B803027404B2
:100FB000B8040274037888F613C238C2394002D2EA
:100FC000384002D2398019C3E54D940C7012755D1A
:100FD000A5755EF1C3E54E9406400B1211CCD2AF5D
:100FE000754E00754D00755D00755E00C230C126FE
:100FF000C2AF51A8E4D2AFE4F559F524F525F53791
:1010000075590812046E1204EF30EDFDA8BDA9BE9B
:10101000E97001F8885A1204F3755908C2AF120535
:101020005A855856855857D2AF303A07C2383031B2
:1010300002D238D228753300120A00120A23120590
:101040006912059912056912059912056912082796
:10105000120922120974120599120817202C031282
:1010600004A9302C031204D912092212099712057F
:10107000991208271209221209BA120599120817A3
:101080001209221209DD12059912082712092212EB
:101090000A001205991204EF120817120922120A07
:1010A000231204F312059930282785585679187AA7
:1010B0000CC3E53399400EC228D2298A358558568B
:1010C000855857800CC3E54F9401400302104D2111
:1010D0005730291F202B1CE535147006C229D22A4F
:1010E000014DF535203A07C3E54F94014003021046
:1010F0004D8064753600203A0F78FA79A4E76002D3
:101100007803C3E55098504FE523604B303A1720E1
:101110003805203107800F303102800A202B07D29A
:101120002B855856017D78F0302B05855856782050
:10113000C3E57198500302104D302B1BC22BC238EF
:10114000303102D238D229753512855856014D05F5
:1011500036E54F6002215A753600C2AF120AA875F3
:101160002500D2AF12047E120AA875240078A4E6E6
:101170006006D290D292D294C3E536940440030222
:101180000C28020DBD901A0D78205105E520B455AC
:101190000AA35105E520B4AA028013755DA5755E0A
:1011A000F1120AB831CC755D00755E00801D901A91
:1011B0000378807B0A5105A308DBFA901A0F788C1C
:1011C0007B1A5105A308DBFA901A2922C2AF5148B5
:1011D0005125901A007402510AA37403510AA37492
:1011E00021510A901A0378807B0A5109A308DBFA7F
:1011F000901A0F788C7B1A5109A308DBFA515B51C6
:1012000039901A2922E493F622E6438F01538FFD89
:10121000FFC3E583941C400122EF855DB7855EB76F
:10122000F0538FFE22438F02438F01855DB7855EA9
:10123000B7901A0DF0538FFC22901A0D7455510A75
:10124000901A0E74AA510A227A3079D07820901A16
:10125000405105E520F709A3DAF7227A3079D090DA
:101260001A40E7510A09A3DAF9227C0512045BDC73
:0B127000FB22C2AF120A45D2AF2222BF
:06148000544C5802030465
:10150000E4F52B757749757816757A10F57BF579C2
:10151000757CD885727D752B00E5E4A2E7B3E5E61E
:0815200092E0F5E60215B42289
:0315300002160B95
:1015500085817685D075E579857AD0857C81D25A6A
:08156000C077C07843E6802249
:10157000305A17C25A85D07AF579D078D0778581DC
:0B1580007C8576818575D085D77B3295
:1015B0000215DE32751CF6751DEB751EE07519BA45
:1015C000751AFEE573751B01B42812751CFC751D98
:1015D000F6751EF1751942751AFF751B0C22C2595A
:1015E000C572F452A4F44280C572C28CC28E758A50
:1015F00000758C007589AA851B8EC289C28BD2AA00
:10160000D2A8C2A9C2BBD28CC23432C2C0C0E030A0
:10161000592AD234E57D428042A4D0E07574A87581
:101620008921538EF0758BFF851A8C85198AC28D9E
:10163000C28FD2BBD28CD28E43A80A32D2AAD2A8F1
:10164000D0E0327B007A0180352059FD2034FA2029
:101650002906202803202000C2AFAB71AA70D2AFA8
:10166000EBC313FBEA13FAEBC313F9EA132AFAE903
:101670003BFBEA24FFEB34FF400474FFFBFAE4FC7D
:10168000C3EB136007FBEA13FA0C80F4EC234B5412
:101690000FC4FBEAC4FA540F4BFBEA54F0FA6BC4D4
:1016A0006B540F4A640FFA78A874E0C0E07416C057
:1016B000E0791C7D17EA540F242B83C0E0C015EAA3
:1016C000C4540F242083C0E0C015EB540F241683AC
:1016D000C0E0C015EBC4540F240B83C0E0C015223A
:1016E0007600D259C149000C1B24303F4B5766721B
:1016F0007C8693A2AFBC0000000000000000000048
:10170000E7F608A61C08A61E08791C22E7F608A61C
:101710001C08A61D08A61C08791C22E7F608A61EB0
:1017200008791D22E7F608A61E08A61C08791C22C7
:10173000E7F608A61C08A61C08A61D08791C22E7C7
:10174000F608A61D08A61D08791C22E7F608A61DA6
:1017500008A61C08791D22E7F608A61D08A61C0885
:10176000A61C08791C22E7F608A61C08A61D087905
:101770001D2209E7F608A61E08791C2209E7F608CB
:10178000A61D08791D2209E7F608A61D08A61C0853
:10179000791C22E7F608A61C08A61C08A61C0879D6
:1017A0001D2209E7F608A61C08A61D08791C2209B7
:1017B000E7F608A61C08A61C08791D2209E7F6080A
:0C17C000A61C08A61C08A61C08791C2208
:1019E0007597DE7597AD43EF02B4A5030219FD901C
:0A19F000FBFDE493B4A5F502FBC073
:1019FD00020B8D020321FFFFFFFFFFFF09FF01FF18
:101A0D0055AA01FFFFFFFFFF03FFFFFF25D0285061
:0D1A1D0004FF02FF7AFF0701FFFF0000FF3A
:101A400023535F4C5F35302320202020202020208E
:101A500023424C48454C492445464D3842313023B9
:101A60002020202020202020202020202020202076
:101C0000C2AFC2D37597DE7597AD7581C075A90057
:101C100075A90043FF80752438752503B1DE752949
:101C2000A5752AF143F12053A4DFD28575D4FF7541
:101C3000E3407DFA780379E67C1075220075230075
:101C4000901DEB7B06752498752501308502814B2C
:101C5000208508D8FBD9F9DCF781BD308508D8FB91
:101C6000D9F9DCF781BDB19EE493A3C39A6004DD8A
:101C7000C381BDDBDBB190600281347B08E493FA61
:101C8000A3B171DBF87A30B171752200752300B110
:101C900090EAFCEBFDC3ED94FE400EB1908A278BD9
:101CA00028ED30E0048A828B83B1907AC270D8C369
:101CB000ED94FE601950CEBD0029EC600F75200038
:101CC0007521FF752900752A000200008100A827F0
:101CD000A9280809D804D90281E0B194EAF281D494
:101CE0000D81A9C3ED94035051EDA2E092007AC595
:101CF000C3E5829400E583941C508C200010438F30
:101D000002438F018529B7852AB7F0300027A8271D
:101D1000A9280809438F01538FFDD804D902A135A2
:101D2000C3E583941C4003A3A11AE28529B7852A41
:101D3000B7F0A3A11A538FFC81857AC1BD030CE4CF
:101D400093A3FAB155DCF8B14D81858187AA22AB06
:101D500023B171EBFAEA6222752608C3E52313F575
:101D600023E52213F52250066323A0632201D52622
:101D7000EAB1DEB1DE75260AEAF4200102D285302E
:101D80000102C285B1DEC3134002C201D526EB2297
:101D9000B194EAFB208502A194308502A1997526B1
:101DA00008AE24AF25C3EF13FFEE13FEB1E2B1DEA0
:101DB000C3EA133085024480FA30E703632201C38B
:101DC000E52313F523E52213F52250066323A063D0
:101DD0002201D526D9E52265236523F52222AE24EA
:101DE000AF250E0FDEFEDFFCD20122424C48656CAF
:091DF0006934373164E8B10601E1
:00000001FF
